:1000000011C020C01FC01EC01DC01CC01BC01AC014
:1000100019C018C017C016C015C014C013C06E6F29
:100020006465200011241FBECFE5D1E0DEBFCDBF47
:1000300010E0A0E6B0E001C01D92A436B107E1F7E0
:100040000BD13CC1DDCFDC01FA0110828C918623FB
:10005000E9F785E88A95F1F788EC90E00197F1F7E8
:100060008C91862319F081E0808301C0108288EC96
:1000700090E00197F1F78C91862319F080818260DE
:10008000808388EC90E00197F1F78C91862319F03A
:1000900080818460808388EC90E00197F1F78C91F7
:1000A000862319F080818860808388EC90E0019736
:1000B000F1F78C91862319F080818061808388EC30
:1000C00090E00197F1F78C91862319F0808180628E
:1000D000808388EC90E00197F1F78C91862319F0EA
:1000E00080818064808388EC90E00197F1F78C91A7
:1000F000862319F080818068808388EC90E00197E6
:10010000F1F785E88A95F1F70895FC018081562F73
:1001100050958523808388EC90E00197F1F7242F98
:10012000332727FD309520FF03C08081862B02C036
:1001300080818523808388EC90E00197F1F721FF8F
:1001400003C08081862B02C080818523808388EC58
:1001500090E00197F1F722FF03C08081862B02C057
:1001600080818523808388EC90E00197F1F723FF5D
:1001700003C08081862B02C080818523808388EC28
:1001800090E00197F1F724FF03C08081862B02C025
:1001900080818523808388EC90E00197F1F725FF2B
:1001A00003C08081862B02C080818523808388ECF8
:1001B00090E00197F1F726FF03C08081862B02C0F3
:1001C00080818523808388EC90E00197F1F747FFD9
:1001D00004C08081862B808303C080815823508394
:1001E00028EC30E0C9010197F1F78081862B8083EC
:1001F000C9010197F1F7C9010197F1F70895EF924D
:10020000FF921F93CF93DF93EA01EE24FF24FE01B8
:10021000149188E390E060E1412F77DF0894E11CBE
:10022000F11C2196112399F710926300F09262005D
:10023000E0926100DF91CF911F91FF90EF900895C0
:10024000C09888EE93E028EC30E0F9013197F1F79F
:100250000197D9F7C09A0895CF93DF9380E886BDC0
:1002600016BCC49ABC98C09AB89AC8ECD0E086E391
:1002700090E068E040E650E0E6DEE2DF809160007A
:100280008233A9F7BC9A88E390E060E14EE150E048
:10029000B6DF88E390E060E14091600036DF88E3FC
:1002A00090E060E14AE031DF88EE93E0FE013197B3
:1002B000F1F70197D9F7C4DFBC98D9CFF894FFCFF5
:00000001FF
